:060000008A118312322870
:08000800A000030E8312A10009
:100010000408A2000A08A30000308A0061228312AB
:100020002208840023088A00210E8300A00E200EDF
:1000300009005B205320432052204F204C204C20AD
:10004000202043204C204F2043204B2020205620AE
:10005000652072202E3131305D20CA0008308A00C0
:10006000002808008312FF30870005080338850048
:100070008316003087000508FC39850083120030A4
:1000800088000508F33985008316FF3088000508CD
:100090000C388500831201308900831600308900F6
:1000A0008312203084008001840A841F5328A030EA
:1000B00084008001840AC0300406031D592883127D
:1000C0000730A900BF30A700FF30A8000B30A50003
:1000D0000130ED000230EC000030F9000630F8008D
:1000E0000030F7000030F6000030FF000730FE005F
:1000F0000030FD000030FC001930E3003C30E4002B
:1001000083168230810083120530900083128C01A7
:10011000831601308C00E0308B0083120314A70D8E
:10012000A80DA90A0A302906031D9B28A901FE3043
:10013000A700FF30A800A220D320A2209621A22051
:100140002C258D288312003087000508FC39850096
:100150008316FF30880005080C38850083124B3069
:100160002907840000088700A630290784000008BA
:10017000E5008500FC3965048500280DA600260DE4
:100180000C39A600270888000508F33926048500E5
:100190002708831688000508F3398312260483167E
:1001A0008500831208008312DB0A5C06E6005B0808
:1001B000DC0066081039031D9529DD0D5D10861AD7
:1001C0005D14DE0D5E10061A5E14DF0D5F108619D9
:1001D0005F14E00D60100619601480305D0603198D
:1001E000FE2880305E060319092980305F06031956
:1001F0003E298030600603195B299529561C022987
:10020000D601952958080E39031D95290130D806C5
:100210009529561C0D29D601952958080C39031D1E
:1002200095290230D800EF01EE01F101F001F30150
:10023000F201E201D814D90A04305906031D22291B
:10024000D901D81000305906031D2929D713EC24F1
:100250003B2901305906031D2F29F0243B29023088
:100260005906031D35290E263B2903305906031D67
:100270003B2900003B291530A5009529561C422931
:10028000D601952958080A39031D952958100430BC
:10029000D80658195029E7011530A500EC249529F6
:1002A000E201EE01EF010330F000F101F201F30190
:1002B0000330E7009529561C5F29D6019529580877
:1002C0000639031D95295810DA0A06305A06031913
:1002D000DA0100305A06031D7029D811EC24952943
:1002E00001305A06031D7829E201D815F324952917
:1002F00002305A06031D8029E201D815F6249529FB
:1003000003305A06031D8729D811EC24952904309F
:100310005A06031D8E29D811EC24952905305A065A
:10032000031D9529D811EC2495290800E10CE10C56
:100330003030E1050608C039E104610801308A0067
:10034000610E8207B829B829B829B829B829B8296F
:10035000B829B829B829B829B829B829B829B52998
:10036000B229B8290130E200B929FF30E200B929E9
:100370000000E2080319602A5818C529D818C729AF
:100380005819252AD819372A602A0000602A013016
:100390005906031DDF2901306206031DD1290724F8
:1003A000D629FF306206031D602A5724E201D717C1
:1003B000E801E901D5018E018F01F024602A0230A5
:1003C0005906031DFB2901306206031DEE29E201D7
:1003D000E30A6308643A0319E301602AFF30620606
:1003E000031D602AE201E3036308FF3A031D602A4C
:1003F0006330E300602A03305906031D602A013090
:100400006206031D112AD717E801E901D5018E0103
:100410008F01EC24E201E40A6408643A0319E40160
:10042000602AFF306206031D602AD717E801E90140
:10043000D5018E018F01EC24E201E4036408FF3A48
:10044000031D602A6330E400602A01306206031D48
:100450002B2AB425302AFF306206031D602ACF25DF
:10046000E201EE01EF010330E700DE25602A000023
:1004700001305A06031D4C2A01306206031D422A30
:100480000D24472AFF306206031D602A5D24E20125
:10049000F401F501F324602A02305A06031D602A94
:1004A00001306206031D562A13245B2AFF306206C0
:1004B000031D602A6324E201FA01FB01F624602A8D
:1004C000080083120C1CE22AD50A10305506031DC1
:1004D000E12AD50164083C3E8E00E708031DE703CE
:1004E000D71FF523013059060319F024D818892A9B
:1004F000D8080319882A03305A060319882A0430B9
:100500005A060319882A05305A060319882A892AA7
:10051000EC246D087906031DAD2A6C087806031DCE
:10052000AD2A6B087706031DAD2A6A087606031DFF
:10053000AD2A69087506031DAD2A68087406031DF7
:10054000AD2A03305A06031DA72AD71656140530C4
:100550005A06031DAD2A571756146D087F06031D52
:10056000D12A6C087E06031DD12A6B087D06031D67
:10057000D12A6A087C06031DD12A69087B06031D5F
:10058000D12A68087A06031DD12A04305A06031DB1
:10059000CB2A5717561405305A06031DD12A571770
:1005A0005614581DE12AE708031DE12A6E086F045E
:1005B00070047104031DDF2A58115614E12AC12565
:1005C000DE250C100B1DCA2B561CF12AD51CF52A52
:1005D000D51DF52A83160030890083120330890661
:1005E000F52A8316033089008312A40A63082406BF
:1005F000031DC92BA4015818672B03305906031992
:10060000982BE708031DB32B2A30840025088407A4
:1006100045300406031D0E2B2A3084000008CB0051
:10062000840A45300406031D172B2A308400000875
:10063000CC00840A45300406031D202B2A30840098
:100640000008CD00840A45300406031D292B2A30FA
:1006500084000008CE00840A45300406031D322BB6
:100660002A3084000008CF00840A45300406031DA8
:100670003B2B2A3084000008D000840A4530040651
:10068000031D442B2A3084000008D100840A453021
:100690000406031D4D2B2A3084000008D200840A72
:1006A00045300406031D562B2A3084000008D30071
:1006B000840A45300406031D5F2B2A30840000089D
:1006C000D400A50A1B3025060319A501C92BCB01AF
:1006D0008030CC00CD0169082D204708CE004808A5
:1006E000CF004908D000D10168082D204708D2006A
:1006F0004808D3004908D400C92B63082F26CB0132
:10070000CC01CD018316360883122D204708CE0078
:100710004808CF004908D000D1018316350883125C
:100720002D204708D2004808D3004908D400C92B1F
:1007300064082F26CB01CC01CD0183163608831225
:100740002D204708CE004808CF004908D000D1012D
:100750008316350883122D204708D2004808D3009D
:100760004908D400C92BCB012830CC00CD01710839
:100770002D204708CE004808CF004908D000D101FD
:1007800070082D204708D2004808D3004908D4003B
:10079000C92B0B110800831684000008B000840ADE
:1007A0000008B100840A0008B200840A0008B300FF
:1007B000840A0008B400840A0008B5008312080007
:1007C0008316840030088000840A31088000840A7F
:1007D00032088000840A33088000840A34088000CC
:1007E000840A35088000831208006830CB2319245E
:1007F0006830E02308007430CB2319247430E023E0
:1008000008007A30CB2319247A30E02308006830BE
:10081000CB2326246830E02308007430CB23262421
:100820007430E02308007A30CB2326247A30E0238A
:1008300008008316B00A0A303006031D3A2CB001B6
:10084000B10A06303106031D3A2CB1018316B20AF3
:100850000A303206031D3A2CB201B30A06303306C1
:10086000031D3A2CB301B40A0A303406031D3A2C96
:10087000B401B50A04303406031D442C0230350699
:10088000031D442CB401B50108006830CB23692452
:100890006830E02308007430CB2369247430E023EF
:1008A00008007A30CB2369247A30E02308006830CE
:1008B000CB2378246830E02308007430CB237824DD
:1008C0007430E02308007A30CB2378247A30E02398
:1008D00008008316B003FF303006031DA22C093038
:1008E000B000B103FF303106031DA22C0530B1006A
:1008F0008316B203FF303206031DA22C0930B2006A
:10090000B303FF303306031DA22C0530B3000030C3
:100910003406031D942C00303506031D942C03303F
:10092000B4000230B500A22CB403FF303406031D1E
:10093000A22C0930B400B503FF303506031DA22CEC
:100940000230B50008006830831684000008BC003F
:10095000840A0008BD00840A0008BE00840A00085A
:10096000BF00840A0008C000840A0008C100831286
:100970008316C601C7010130C80001304106031DBE
:10098000C32C0A30C60702304106031DC92C14309F
:10099000C6074008C60718304602C700031DD32CFF
:1009A000C101C101EA2C0C304602C700031DDA2C3C
:1009B000C814EA2C0C304602C700031CEA2CC10103
:1009C000C0010A304702031CE72CC700C10A4708D0
:1009D000C000C81483120800A324C1308400F92C7D
:1009E0006D308400F92C79308400F92C7F3084003C
:1009F000F92C00082D204708AA004808AB00490838
:100A0000AC00AD010008031D092DAA01AB01AC012A
:100A1000AD01840300082D204708AE004808AF0050
:100A20004908B000B1012830B200B30184030008C6
:100A30002D204708B4004808B5004908B600B701A2
:100A4000840300082D204708B8004808B900490869
:100A5000BA00BB01BC0108008316A601A701A801CA
:100A6000A901AA01AB01AC01AD01AE01AF01831236
:100A7000D9080319532D8316A614A714A81483129A
:100A8000A63084000130590603190014A7308400F1
:100A90000230590603190014A830840003305906A7
:100AA00003190014732DE601A63084008316481C38
:100AB0005D2DC818001480145F2D0014801483125B
:100AC000660869060319672DE60A840A562D681C14
:100AD000732D8316481C702DC81800108010722DBD
:100AE000001080108312AD308400581D792D001441
:100AF000801401305A0603198E2D02305A0603194C
:100B0000922D03305A060319962D04305A06031904
:100B10009B2D05305A060319A02DA72D83162E14E0
:100B20008312A72D83162F148312A72D83162E143C
:100B3000AE148312A72D83162F14AF148312A72D82
:100B400083162E14AE142F14AF148312A72D080091
:100B5000EE0A0A306E06031DC02DEE01EF0A0630C4
:100B60006F06031DC02DEF01F00A0A307006031D49
:100B7000C02DF001F10A0A307106031DC02DF101EC
:100B80000800EE03FF306E06031DDD2D0930EE0078
:100B9000EF03FF306F06031DDD2D0530EF00F0037E
:100BA000FF307006031DDD2D0930F000F103FF302A
:100BB0007106031DDD2D0930F100080071082D209C
:100BC0004708AA004808AB004908AC00AD0171080D
:100BD000031DEE2DAA01AB01AC01AD0170082D2063
:100BE0004708AE004808AF004908B000B1018030A6
:100BF000B200B3016F082D204708B4004808B500C3
:100C00004908B600B7016E082D204708B80048080B
:100C1000B9004908BA00BB01BC0108001030AA00A5
:100C20003830AB007C30AC00FE30AD003830AE0068
:100C30003830AF003830B0002830B100B201B30115
:100C4000B401B501B601B701B801B901BA01BB01E0
:100C5000BC01080083160030B4006430B300831672
:100C6000B300B4010F30B900B701B601B5010310EC
:100C7000B30DB40DB50DB60DB70D03303507B80083
:100C8000B819B50030303507B800B81BB5000330CF
:100C90003607B800B819B60030303607B800B81BB0
:100CA000B60003303707B800B819B700303037073F
:100CB000B800B81BB700B90B382EB30DB40DB50D85
:100CC000B60DB70D350E0F39B60035080F39B50022
:040CD0008312080083
:1010000008308A000310CA0DCA0D4A0D8207FE304F
:10101000C7008230C800FE30C90000005728843065
:10102000C700FE30C8008030C90000005728E230F9
:10103000C7009230C8008E30C90000005728923097
:10104000C7009230C800FE30C900000057281E308B
:10105000C7001030C800FE30C900000057288E308D
:10106000C7008A30C800FA30C90000005728FE3097
:10107000C7009230C800F030C90000005728023085
:10108000C7000230C800FE30C90000005728FE30FB
:10109000C7009230C800FE30C900000057281E303B
:1010A000C7009230C800FE30C900000057288A11DE
:0210B000080036
:02400E00B13FC0
:00000001FF
